:060000000A128A11122809
:10000800FE00030EF1000408F2000A08F300831250
:1000180003137F08F4000A168A15A02F0A168A15FA
:10002800B12E831603179A111A121412171294116B
:1000380091111112BA299415941923282728831687
:10004800031791152A28831603179111482F17169D
:10005800171A2F28332883160317141636288316E1
:1000680003171412141A39283D28831603179A15F2
:100078004028831603179A119A194328472883168C
:10008800031791154A2883160317911191194D28C2
:1000980051288316031711165428831603171112B3
:1000A800482F1716171A59285D2883160317941511
:1000B80060288316031794119419632867288316F8
:1000C80003179A156A28831603179A119A196D2827
:1000D8007128831603179115742883160317911135
:1000E800911977287B288316031711167E28831603
:1000F80003171112482F94159419832887288316FB
:10010800031791158A2883160317911191198D28C1
:100118009128831603179A159428831603179A11A2
:100128009A1997289B28831603171A169E28831650
:1001380003171A12482F1716171AA328A728831669
:1001480003179415AA288316031794119419AD2838
:10015800B128831603179A15B428831603179A1122
:100168009A19B728BB28831603171A16BE288316B0
:1001780003171A121A1AC128C5288316031711164D
:10018800C828831603171112482F9A159A19CD28D3
:10019800D128831603179415D428831603179411AE
:1001A8009419D728DB28831603171716DE28831619
:1001B80003171712171AE128E528831603171416D0
:1001C800E828831603171412141AEB28EF2883164D
:1001D80003171A16F228831603171A121A1AF52883
:1001E800F928831603171116FC2883160317111212
:1001F800482F941594190129052983160317911579
:10020800082983160317911191190B290F298316B1
:10021800031711161229831603171112482F9A155E
:100228009A1917291B29831603171A161E298316CC
:1002380003171A121A1A21292529831603171416C7
:100248002829831603171412141A2B292F29831609
:10025800031717163229831603171712171A352989
:1002680039298316031794153C298316031794110B
:1002780094193F2943298316031791154629831694
:1002880003179111911949294D298316031711163E
:100298005029831603171112482F9A159A195529B0
:1002A8005929831603171A165C29831603171A127D
:1002B8001A1A5F29632983160317171666298316E6
:1002C80003171712171A69296D298316031794152E
:1002D80070298316031794119419732977298316A3
:1002E800031791157A2983160317911191197D29FE
:1002F80081298316031711168429831603171112EF
:10030800482F1A161A1A89298D29831603171416C5
:100318009029831603171412141A93299729831600
:10032800031717169A29831603171712171A9D29E8
:10033800A129831603179415A4298316031794116A
:100348009419A729AB29831603179115AE2983168B
:10035800031791119119B129B5298316031711169D
:10036800B829831603171112482F482F7508003A29
:1003780003198529013A03191F28033A03192B2861
:10038800013A03195528073A03197F28013A031936
:100398009F28033A0319C928013A0319FD280F3A7F
:1003A80003191329013A03195129482F482F831695
:1003B8000317131093109910901019101610961017
:1003C800802B19141918E929ED2983160317161417
:1003D800F029831603171610482F90149018F52942
:1003E800F929831603179914FC2983160317991002
:1003F8009918FF29032A831603171314062A83164C
:10040800031713101318092A0D2A83160317161435
:10041800102A8316031716101618132A172A83167C
:10042800031796141A2A831603179610482F901448
:1004380090181F2A232A831603171914262A8316AD
:10044800031719101918292A2D2A831603171314AC
:10045800302A8316031713101318332A372A8316E2
:10046800031716143A2A83160317161016183D2A6E
:10047800412A831603179614442A831603179610E5
:10048800482F19141918492A4D2A831603171614C8
:10049800502A8316031716101618532A572A83163C
:1004A800031713145A2A83160317131013185D2AF7
:1004B800612A831603179314642A8316031793106B
:1004C800482F90149018692A6D2A83160317191457
:1004D800702A8316031719101918732A772A831696
:1004E800031713147A2A83160317131013187D2A77
:1004F800812A831603179314842A831603179310EB
:100508009318872A8B2A8316031796148E2A831624
:1005180003179610482F13141318932A972A831633
:10052800031719149A2A83160317191019189D2AE4
:10053800A12A831603179014A42A83160317901070
:100548009018A72AAB2A831603179914AE2A831684
:10055800031799109918B12AB52A8316031793140B
:10056800B82A8316031793109318BB2ABF2A831639
:1005780003179614C22A831603179610482F1914C6
:100588001918C72ACB2A831603171614CE2A8316DE
:10059800031716101618D12AD52A8316031796148E
:1005A800D82A831603179610482F13141318DD2A18
:1005B800E12A831603179314E42A8316031793106A
:1005C8009318E72AEB2A831603179914EE2A831641
:1005D800031799109918F12AF52A8316031790140E
:1005E800F82A8316031790109018FB2AFF2A8316FF
:1005F80003171914022B8316031719101918052B42
:10060800092B8316031716140C2B831603171610C1
:1006180016180F2B132B831603179614162B8316F5
:1006280003179610482F131413181B2B1F2B831610
:1006380003179314222B8316031793109318252B53
:10064800292B8316031790142C2B8316031790104D
:1006580090182F2B332B831603171914362B831658
:10066800031719101918392B3D2B83160317161465
:10067800402B8316031716101618432B472B831687
:10068800031796144A2B831603179610482F9314B2
:1006980093184F2B532B831603179914562B831635
:1006A800031799109918592B5D2B8316031790146B
:1006B800602B8316031790109018632B672B8316F3
:1006C800031719146A2B83160317191019186D2BA1
:1006D800712B831603171614742B83160317161021
:1006E8001618772B7B2B8316031796147E2B8316ED
:1006F80003179610482F482F7508003A03194B2BFB
:10070800013A0319E529033A0319F129013A0319B2
:100718001B2A073A0319452A013A0319652A033A9D
:1007280003198F2A013A0319C32A0F3A0319D92A40
:10073800013A0319172B482F482F831203179311D7
:10074800131119111011991196111611462D991599
:100758009919AF2BB32B831203179615B62B831257
:1007680003179611482F10151019BB2BBF2B831296
:1007780003171915C22B8312031719111919C52B41
:10078800C92B831203179315CC2B831203179311CC
:100798009319CF2BD32B831203179615D62B8312BD
:1007A800031796119619D92BDD2B831203171615EB
:1007B800E02B831203171611482F10151019E52B7B
:1007C800E92B831203179915EC2B83120317991140
:1007D8009919EF2BF32B831203179315F62B83121A
:1007E800031793119319F92BFD2B831203179615F1
:1007F800002C8312031796119619032C072C8312C9
:10080800031716150A2C831203171611482F99156A
:1008180099190F2C132C831203179615162C831273
:10082800031796119619192C1D2C8312031793156B
:10083800202C8312031793119319232C272C83122E
:10084800031713152A2C831203171311482F101599
:1008580010192F2C332C831203179915362C831259
:10086800031799119919392C3D2C831203179315E5
:10087800402C8312031793119319432C472C83128E
:10088800031713154A2C83120317131113194D2C30
:10089800512C831203171615542C831203171611A3
:1008A800482F93159319592C5D2C8312031799150A
:1008B800602C8312031799119919632C672C8312E2
:1008C800031710156A2C83120317101110196D2CB9
:1008D800712C831203171915742C8312031719111D
:1008E8001919772C7B2C8312031713157E2C83126E
:1008F800031713111319812C852C8312031716154E
:10090800882C831203171611482F991599198D2CC5
:10091800912C831203179615942C831203179611A2
:100928009619972C9B2C8312031716159E2C83124D
:1009380003171611482F93159319A32CA72C83126C
:1009480003171315AA2C8312031713111319AD2CAF
:10095800B12C831203171915B42C8312031719111C
:100968001919B72CBB2C831203171015BE2C831230
:10097800031710111019C12CC52C831203179915D0
:10098800C82C8312031799119919CB2CCF2C8312D9
:1009980003179615D22C8312031796119619D52C86
:1009A800D92C831203171615DC2C83120317161182
:1009B800482F93159319E12CE52C8312031713156F
:1009C800E82C8312031713111319EB2CEF2C831245
:1009D80003171015F22C8312031710111019F52C98
:1009E800F92C831203179915FC2C831203179911FC
:1009F8009919FF2C032D831203179615062D8312C0
:100A0800031796119619092D0D2D83120317161524
:100A1800102D831203171611482F13151319152DAE
:100A2800192D8312031719151C2D83120317191179
:100A380019191F2D232D831203171015262D831224
:100A4800031710111019292D2D2D8312031799152D
:100A5800302D8312031799119919332D372D8312CD
:100A6800031796153A2D83120317961196193D2DE3
:100A7800412D831203171615442D831203171611DF
:100A8800482F482F7508003A0319112D013A031908
:100A9800AB2B033A0319B72B013A0319E12B073A99
:100AA80003190B2C013A03192B2C033A0319552C63
:100AB800013A0319892C0F3A03199F2C013A03199B
:100AC800DD2C482F482F8312031793121312191283
:100AD80010129912961216120C2F9916991A752D32
:100AE800792D8312031796167C2D831203179612FD
:100AF800482F1016101A812D852D831203171916E9
:100B0800882D831203171912191A8B2D8F2D831212
:100B180003179316922D831203179312931A952D88
:100B2800992D8312031796169C2D8312031796127C
:100B3800961A9F2DA32D831203171616A62D83121E
:100B480003171612482F1016101AAB2DAF2D83124B
:100B580003179916B22D831203179912991AB52DF6
:100B6800B92D831203179316BC2D83120317931202
:100B7800931ABF2DC32D831203179616C62D831201
:100B880003179612961AC92DCD2D83120317161620
:100B9800D02D831203171612482F9916991AD52D9E
:100BA800D92D831203179616DC2D8312031796127C
:100BB800961ADF2DE32D831203179316E62D831261
:100BC80003179312931AE92DED2D831203171316A9
:100BD800F02D831203171312482F1016101AF52D33
:100BE800F92D831203179916FC2D831203179912F6
:100BF800991AFF2D032E831203179316062E8312BC
:100C080003179312931A092E0D2E83120317131626
:100C1800102E831203171312131A132E172E831272
:100C2800031716161A2E831203171612482F931637
:100C3800931A1F2E232E831203179916262E83121A
:100C480003179912991A292E2D2E8312031710169D
:100C5800302E831203171012101A332E372E8312D8
:100C6800031719163A2E831203171912191A3D2E53
:100C7800412E831203171316442E831203171312DF
:100C8800131A472E4B2E8312031716164E2E831255
:100C980003171612482F9916991A532E572E831296
:100CA800031796165A2E831203179612961A5D2E5C
:100CB800612E831203171616642E83120317161259
:100CC800482F9316931A692E6D2E83120317131645
:100CD800702E831203171312131A732E772E831292
:100CE800031719167A2E831203171912191A7D2E53
:100CF800812E831203171016842E831203171012E5
:100D0800101A872E8B2E8312031799168E2E831294
:100D180003179912991A912E952E83120317961676
:100D2800982E831203179612961A9B2E9F2E8312C3
:100D380003171616A22E831203171612482F93169E
:100D4800931AA72EAB2E831203171316AE2E8312F7
:100D580003171312131AB12EB52E83120317101688
:100D6800B82E831203171012101ABB2EBF2E83122F
:100D780003179916C22E831203179912991AC52EB2
:100D8800C92E831203179616CC2E831203179612B8
:100D9800961ACF2ED32E831203171616D62E831229
:100DA80003171612482F1316131ADB2EDF2E831281
:100DB80003171916E22E831203171912191AE52EB2
:100DC800E92E831203171016EC2E83120317101244
:100DD800101AEF2EF32E831203179916F62E83128C
:100DE80003179912991AF92EFD2E831203179616D6
:100DF800002F831203179612961A032F072F8312B8
:100E0800031716160A2F831203171612482F482F96
:100E18007508003A0319D72E013A0319712D033AC0
:100E280003197D2D013A0319A72D073A0319D12D6E
:100E3800013A0319F12D033A03191B2E013A03193C
:100E48004F2E0F3A0319652E013A0319A32E482F86
:100E5800482F482F7608013A03194C2F033A0319F3
:100E6800522F013A0319552F073A03195E2F013AF9
:100E780003191528033A0319DB29013A0319A12B91
:100E88000F3A0319672D482F08000A168A11C22F36
:100E98000A168A11C02E0A168A115B2D0A168A11A3
:100EA800EF2C0A128A15A6290A168A117C2E0A1610
:100EB8008A11322C0A168A11E82B64308312031324
:100EC800A4000030A5002D08A701A7072C08A6013B
:100ED800A6070A168A110C200A128A118312031314
:100EE8002408AE002E08B2003208AE00AF012E086A
:100EF800A0002F08A1006430A2000030A3000A1649
:100F08008A1516270A128A11831203132009B000C2
:100F18002109B100B00A0319B10A2C083007AC0046
:100F28002D0803182D0A3107AD003208AE002E082F
:100F3800F50006300A168A11BC260A128A110A30F0
:100F480083120313A4000030A5002D08A701A707EA
:100F58002C08A601A6070A168A110C200A128A1163
:100F6800831203132408AE002E08B2003208AE0024
:100F78002E08F50007300A168A11BC260A128A11B3
:100F8800831203133208AE00AF012E08A0002F0809
:100F9800A1000A30A2000030A3000A168A151627FD
:100FA8000A128A11831203132009B0002109B10023
:100FB800B00A0319B10A2C083007AC002D08031831
:100FC8002D0A3107AD002C08AE002E08F5000830B8
:100FD8000A168A11BC260A128A11831603171715D6
:020FE8000800FF
:10100200831203131F150A168A15C1260A128A159E
:101012000A168A15C1260A128A15831203139F140F
:1010220012289F1815281628122817281E08B30000
:10103200B4013308B400B301831603131E088312EC
:1010420003133307BE000030031801303407BF001A
:101052000A30A4000030A5003E08D13EA0003F089F
:101062000318013EFE3EA1002430A2000030A3007E
:101072000A168A1516270A128A15831203132108E3
:10108200A701A7072008A601A6070A168A110C20A5
:101092000A128A15831203132508BF01BF07240809
:1010A200BE01BE07831203179015831203133F0874
:1010B200AD01AD073E08AC01AC070A128A116127E7
:1010C2000A128A1508009816981A68286C28831242
:1010D200031715176F28831203171513151B722890
:1010E2007628831203171B177928831203171B1301
:1010F2001B1B7C288028831203179B1683288312CC
:1011020003179B129B1A86288A28831203179216AA
:101112008D288312031792120A128A11482F1B1765
:101122001B1B942898288312031715179B288312D8
:1011320003171513151B9E28A2288312031798164E
:10114200A528831203179812981AA828AC2883128C
:1011520003179516AF28831203179512951AB22812
:10116200B628831203179B16B928831203179B1202
:101172009B1ABC28C028831203179216C328831215
:10118200031792128D281517151BC828CC28831215
:1011920003171217CF28831203171213121BD22818
:1011A200D628831203179216D92883120317921294
:1011B2008D281B171B1BDE28E228831203179B16A0
:1011C200E528831203179B129B1AE828EC28831246
:1011D20003179516EF28831203179512951AF22812
:1011E200F628831203179816F92883120317981208
:1011F200981AFC2800298312031715170329831252
:1012020003171513151B06290A2983120317121730
:101212000D29831203171213121B1029142983128A
:101222000317921617298312031792128D281B1780
:101232001B1B1C292029831203179B1623298312A7
:1012420003179B129B1A26292A2983120317981621
:101252002D29831203179812981A302934298312E0
:10126200031715173729831203171513151B3A296C
:101272003E298312031712174129831203171213EF
:10128200121B442948298312031792164B298312F1
:10129200031792128D289B169B1A502954298312E8
:1012A200031795165729831203179512951A5A296F
:1012B2005E29831203179816612983120317981265
:1012C200981A642968298312031715176B29831248
:1012D20003171513151B6E29722983120317121790
:1012E2007529831203171213121B78297C29831282
:1012F200031792167F298312031792128D288D28C5
:101302007508003A03194C29013A0A168A11031981
:10131200FB2C033A0319072D013A0319312D0A1246
:101322008A15073A0319B829013A03196428033ABE
:1013320003199028013A0319C4280F3A0319DA282D
:10134200013A031918298D288D28831603171A13B9
:10135200831203179B139513981383160317141301
:1013620011138312031792130A168A11C32B0A123E
:101372008A114F2F831603179416941AC129C5296F
:10138200831603179116C829831603179112911A0F
:10139200CB29CF29831603179A16D229831603174E
:1013A2009A129A1AD529D929831203171A15DC29F8
:1013B200831203171A110A128A11482F17151719C7
:1013C200E329E729831603179416EA2983160317DC
:1013D2009412941AED29F129831603179A16F42907
:1013E200831603179A129A1AF729FB2983120317F5
:1013F2001A15FE29831203171A111A19012A052A2E
:10140200831203171115082A831203171111DC29FD
:10141200831603179A169A1A0F2A132A831603178A
:101422009416162A831603179412941A192A1D2A3F
:10143200831203171715202A83120317171117197E
:10144200232A272A8312031714152A2A8312031721
:10145200141114192D2A312A831203171A15342A4A
:10146200831203171A111A19372A3B2A83120317F8
:1014720011153E2A831203171111DC298316031753
:101482009416941A452A492A8316031791164C2A50
:10149200831603179112911A4F2A532A83120317A4
:1014A2001115562A831203171111DC29831603170B
:1014B2009A169A1A5D2A612A831203171A15642A48
:1014C200831203171A111A19672A6B2A8312031738
:1014D20014156E2A8312031714111419712A752A0E
:1014E200831203171715782A831203171711171976
:1014F2007B2A7F2A831603179416822A83160317E0
:101502009412941A852A892A8316031791168C2A13
:10151200831603179112911A8F2A932A83120317A3
:101522001115962A831203171111DC29831603174A
:101532009A169A1A9D2AA12A831203171A15A42A07
:10154200831203171A111A19A72AAB2A8312031737
:101552001715AE2A8312031717111719B12AB52AC4
:10156200831603179416B82A831603179412941A33
:10157200BB2ABF2A831603179116C22A83160317A2
:101582009112911AC52AC92A831203171115CC2A5E
:10159200831203171111DC291A151A19D12AD52A17
:1015A200831203171415D82A83120317141114195E
:1015B200DB2ADF2A831203171715E22A8312031785
:1015C20017111719E52AE92A831603179416EC2A2C
:1015D200831603179412941AEF2AF32A8316031719
:1015E2009116F62A831603179112911AF92AFD2AE7
:1015F200831203171115002B831203171111DC2913
:10160200DC297508003A0319CD2A013A0A168A1113
:101612000319FA2B033A0319082C0A128A15013A04
:101622000319272B073A0319BB29013A0319DF29AA
:10163200033A0319092A013A03193F2A0F3A0319F7
:10164200572A013A0319972ADC29DC290A128A113E
:101652005B2F83120313AA002A08A6002608A900FA
:101662000B302A02031C362B372B672D0A30A000C1
:101672000030A1002A08A600A7012608A200270818
:10168200A3000A168A115C200A128A158312031318
:101692002008A8002808A900672D672D83160317C4
:1016A2001616161A552B592B8316031796155C2BF3
:1016B20083160317961196195F2B632B8316031754
:1016C2001615662B8316031716111619692B6D2B27
:1016D200831603171315702B83160317131113198F
:1016E200732B772B8316031719157A2B831603177F
:1016F200191119197D2B812B831603171015842BB1
:101702008316031710111019872B8B2B83160317BF
:1017120099158E2B8316031799119919912B952BD5
:10172200831603171916982B831603171912191A01
:101732009B2B9F2B831603171316A22B83160317BB
:101742001312131AA52BA92B831603179315AC2B6F
:10175200831603179311892D8316031796151612F4
:101762001611131119111011991119121312931143
:10177200892D8316031716151619C02BC42B831631
:1017820003179615C72B83160317961116121311FA
:10179200191110119911191213129311892D83160F
:1017A200031713151319D62BDA2B831603171615E5
:1017B200DD2B8316031716111619E02BE42B831663
:1017C20003179615E72B8316031796111612191194
:1017D20010119911191213129311892D83160317DF
:1017E20019151919F52BF92B831603171315FC2B51
:1017F2008316031713111319FF2B032C83160317D8
:101802001615062C8316031716111619092C0D2C02
:10181200831603179615102C8316031796111612AA
:1018220010119911191213129311892D831603178E
:10183200101510191D2C212C831603171915242C91
:101842008316031719111919272C2B2C831603172A
:1018520013152E2C8316031713111319312C352C43
:10186200831603171615382C83160317161116192B
:101872003B2C3F2C831603179615422C8316031715
:10188200961116129911191213129311892D83169A
:101892000317991599194E2C522C831603171015FC
:1018A200552C8316031710111019582C5C2C831613
:1018B200031719155F2C8316031719111919622CB6
:1018C200662C831603171315692C8316031713113D
:1018D20013196C2C702C831603171615732C831690
:1018E200031716111619762C7A2C831603179615E0
:1018F2007D2C8316031796111612191213129311C7
:10190200892D831603171916191A882C8C2C831605
:10191200031799158F2C8316031799119919922C75
:10192200962C831603171015992C83160317101182
:1019320010199C2CA02C831603171915A32C83169F
:10194200031719111919A62CAA2C8316031713159C
:10195200AD2C8316031713111319B02CB42C831654
:1019620003171615B72C8316031716111619BA2C5E
:10197200BE2C831603179615C12C831603179611D6
:10198200161213129311892D831603171316131AA5
:10199200CB2CCF2C831603171916D22C83160317C0
:1019A2001912191AD52CD92C831603179915DC2C68
:1019B2008316031799119919DF2CE32C8316031749
:1019C2001015E62C8316031710111019E92CED2CB3
:1019D200831603171915F02C8316031719111919F9
:1019E200F32CF72C831603171315FA2C83160317FF
:1019F20013111319FD2C012D831603171615042D2F
:101A02008316031716111619072D0B2D83160317AC
:101A120096150E2D83160317961116129311892D02
:101A2200831603171616161A172D1B2D8316031766
:101A320013161E2D831603171312131A212D252D8B
:101A4200831603171916282D831603171912191A4C
:101A52002B2D2F2D831603179915322D831603175D
:101A620099119919352D392D8316031710153C2D0F
:101A720083160317101110193F2D432D83160317D8
:101A82001915462D8316031719111919492D4D2DB4
:101A9200831603171315502D8316031713111319E9
:101AA200532D572D8316031716155A2D8316031718
:101AB200161116195D2D612D831603179615642DC7
:101AC2008316031796119311892D892D83120313FF
:101AD2002908003A03194F2B013A0319AD2B033A97
:101AE2000319BA2B013A0319D02B073A0319EF2B2A
:101AF200013A0319172C033A0319482C013A031926
:101B0200822C0F3A0319C52C013A0319112D892D84
:101B12000800F500BE2F83160317181015101B10AE
:101B2200121092109B10951098108312031797139E
:101B320094139A13911312101B1015101810981069
:101B420095109B109210FF2F831203179214831685
:101B52000317181015101B10121092109B109510DD
:101B6200981083120317971394139A139113121058
:101B72001B1015101810981095109B10FF2F831230
:101B820003179B14921483160317181015101B10B9
:101B9200121092109B10951098108312031797132E
:101BA20094139A13911312101B10151018109810F9
:101BB2009510FF2F8312031795149B14921483160A
:101BC2000317181015101B10121092109B1095106D
:101BD200981083120317971394139A1391131210E8
:101BE2001B10151018109810FF2F8312031798144A
:101BF20095149B14921483160317181015101B10BA
:101C0200121092109B1095109810831203179713BD
:101C120094139A13911312101B1015101810FF2F02
:101C2200831203171814981495149B149214831694
:101C32000317181015101B10121092109B109510FC
:101C4200981083120317971394139A139113121077
:101C52001B101510FF2F8312031715141814981454
:101C620095149B14921483160317181015101B1049
:101C7200121092109B10951098108312031797134D
:101C820094139A13911312101B10FF2F8312031730
:101C92001B1415141814981495149B14921483167B
:101CA2000317181015101B10121092109B1095108C
:101CB200981083120317971394139A139113121007
:101CC200FF2F8312031712141B14151418149814DF
:101CD20095149B14921483160317181015101B10D9
:101CE200121092109B1095109810831203179713DD
:101CF20094139A139113FF2F83120317911712143F
:101D02001B1415141814981495149B14921483160A
:101D12000317181015101B10121092109B1095101B
:101D2200981083120317971394139A13FF2F831299
:101D320003179A17911712141B14151418149814D8
:101D420095149B14921483160317181015101B1068
:101D5200121092109B10951098108312031797136C
:101D62009413FF2F8312031794179A1791171214C3
:101D72001B1415141814981495149B14921483169A
:101D82000317181015101B10121092109B109510AB
:101D92009810831203179713FF2F831203179717B5
:101DA20094179A17911712141B14151418149814D7
:101DB20095149B14921483160317181015101B10F8
:101DC200121092109B1095109810FF2F8316031774
:101DD200981483120317971794179A1791171214CE
:101DE2001B1415141814981495149B14921483162A
:101DF2000317181015101B10121092109B1095103B
:101E0200FF2F83160317951498148312031797173D
:101E120094179A17911712141B1415141814981466
:101E220095149B14921483160317181015101B1087
:101E3200121092109B10FF2F831603179B149514F8
:101E4200981483120317971794179A17911712145D
:101E52001B1415141814981495149B1492148316B9
:101E62000317181015101B1012109210FF2F831653
:101E7200031792149B14951498148312031797173F
:101E820094179A17911712141B14151418149814F6
:101E920095149B14921483160317181015101B1017
:101EA2001210FF2F83160317121492149B14951409
:101EB200981483120317971794179A1791171214ED
:101EC2001B1415141814981495149B149214831649
:101ED2000317181015101B10FF2F831603171B145E
:101EE200121492149B1495149814831203179717C3
:101EF20094179A17911712141B1415141814981486
:101F020095149B1492148316031718101510FF2FA3
:101F12008316031715141B14121492149B14951490
:101F2200981483120317971794179A17911712147C
:101F32001B1415141814981495149B1492148316D8
:101F420003171810FF2F83160317181415141B14E8
:101F5200121492149B149514981483120317971752
:101F620094179A17911712141B1415141814981415
:101F720095149B149214FF2FFF2F7508003A031932
:101F82008C2D013A0319A52D033A0319C02D013AEC
:101F92000319DB2D073A0319F62D013A0319112E05
:101FA200033A03192C2E013A0319472E0F3A03194B
:101FB200622E013A03197D2E033A0319982E013A33
:101FC2000319B32E073A0319CE2E013A0319E72E4D
:101FD200033A0319022F013A03191D2F1F3A03195D
:101FE200382F013A0319532F033A03196E2F013A7E
:0E1FF2000319892F073A0319A42FFF2F0800A7
:1020180083120313A901AA0125082404031915280A
:1020280016285428AB010314AB0D262801300310E1
:10203800A40DA50DFF3E031D1B280130A80028088C
:10204800AB072628A51F29282A281A282C282C2837
:1020580001300310A90DAA0DFF3E031D2D282508E8
:102068002702031D392824082602031C3C283D2882
:1020780045282408A6022508031CA703A70229143B
:10208800452801300310A50CA40CFF3E031D46286B
:102098000130AB02031D512852282C2854285428FB
:1020A8002A08A501A5072908A401A4075B28080098
:1020B80083120313A501A31F622863286C28A209B1
:1020C800A309A20A0319A30AA5010314A50D6C28E4
:1020D800A11F6F2870287628A009A109A00A031952
:1020E800A10A76282108200403197B287C28B22815
:1020F800A4010314A40D8C2801300310A00DA10D18
:10210800FF3E031D81280130F5007508A4078C28BF
:10211800A11F8F289028802892289228210823021E
:10212800031D982820082202031C9B289C28A3280A
:102138002008A2022108031CA303A302A32801303C
:102148000310A10CA00CFF3E031DA4280130A4021B
:10215800031DAF28B0289228B228B2282508031DED
:10216800B628BC28A209A309A20A0319A30ABC28F5
:102178002308A101A1072208A001A007C32808007D
:102188008312031341080A168A15D9260A168A11DA
:102198000A30831203134102031CD328D428EB28E6
:1021A8003D08AB002B08F50001300A168A11BC2641
:1021B8000A168A11831203133B08AB002B08F5009B
:1021C80002300A168A11BC260A168A1104290A3016
:1021D80083120313AB002B08F50001300A168A118D
:1021E800BC260A168A11831203133B08AB002B087E
:1021F800F50002300A168A11BC260A168A1104292B
:10220800831203133A080A168A15D9260A168A1160
:10221800831203133D08AB002B08F50003300A16A0
:102228008A11BC260A168A11831203133B08AB00D5
:102238002B08F50004300A168A11BC260A168A11E2
:10224800831203133C080A128A152A230A168A11D4
:102258000800831203131F110A168A15C1260A16CD
:102268008A11831203139F1439299F183C293D2989
:1022780039293E291E08B300B4013308B400B3015C
:10228800831603131E08831203133307B6000030A6
:10229800031801303407B7003708A101A107360831
:1022A800A001A0071E30A2000030A3000A168A155C
:1022B80016270A168A11831203132108B701B707D4
:1022C8002008B601B6070A30A4000030A500370878
:1022D800A701A7073608A601A6070A168A110C2027
:1022E8000A168A11831203132508B701B7072408B1
:1022F800B601B6073708AD01AD073608AC01AC0723
:102308000A168A11A9210A168A1196308312031314
:10231800A4000030A5003708A701A7073608A601C2
:10232800A6070A168A110C200A168A1183120313AB
:102338002508B701B7072408B601B60736080A12F8
:102348008A158A250A168A110800E83083120313B1
:10235800A4000330A5002D08A701A7072C08A60193
:10236800A6070A168A110C200A168A11831203136B
:102378002408AE002E08B2003208AE002E08F50080
:1023880002300A168A11BC260A168A118312031310
:102398003208AE00AF012E08A0002F08A100E830D7
:1023A800A2000330A3000A168A1516270A168A11F6
:1023B800831203132009B0002109B100B00A0319E0
:1023C800B10A2C083007AC002D0803182D0A310774
:1023D800AD006430A4000030A5002D08A701A707B0
:1023E8002C08A601A6070A168A110C200A168A11BB
:1023F800831203132408AE002E08B2003208AE0080
:102408002E08F50003300A168A11BC260A168A110E
:10241800831203133208AE00AF012E08A0002F0864
:10242800A1006430A2000030A3000A168A151627FE
:102438000A168A11831203132009B0002109B1007A
:10244800B00A0319B10A2C083007AC002D0803188C
:102458002D0A3107AD000A30A4000030A5002D0870
:10246800A701A7072C08A601A6070A168A110C209F
:102478000A168A11831203132408AE002E08B2002C
:102488003208AE002E08F50004300A168A11BC2660
:102498000A168A11831203133208AE00AF012E0800
:1024A800A0002F08A1000A30A2000030A3000A16DD
:1024B8008A1516270A168A11831203132009B000F9
:1024C8002109B100B00A0319B10A2C083007AC0081
:1024D8002D0803182D0A3107AD002C08AE002E0870
:1024E800F50005300A168A11BC260A168A1108005A
:1024F8000A168A1542270A168A11D52AD52A83125E
:10250800031718151817771C8A2A8B2A922A0A1675
:102518008A11C4200A168A117710922A831203138B
:102528003808013A031D992A9A2AAA2A0230B500C6
:102538003508C000B8010A168A15F5260A168A1148
:102548000A168A15C1260A168A11AA2A83120313A3
:102558003908013A031DB12AB22AD52A0130B5003B
:102568003508BA073A083C3A031DBB2ABC2ACC2ACC
:10257800BA010130B5003508C1070D304102031C0E
:10258800C62AC72ACC2AC1010314C10DCC2ACC2AD9
:10259800B90177140A168A15C1260A168A11D52A8E
:1025A800D52A831203134008013A0319DC2ADD2ACD
:1025B800832A0F2B0F2B8312031715150A168A115E
:1025C8002D210A168A11831203133808013A031DB4
:1025D800EE2AEF2AFF2A0330B5003508C000B801FB
:1025E8000A168A15F5260A168A110A168A15C126A8
:1025F8000A168A11FF2A831203133908013A031DA8
:10260800062B072B0F2BB9010A168A15C1260A16A5
:102618008A110F2B0F2B831203134008023A031958
:10262800162B172BDF2A482B482B831203171B1551
:102638000A128A1501200A168A1183120313380810
:10264800013A031D282B292B382BC0010314C00D78
:10265800B8010A168A15F5260A168A110A168A1565
:10266800C1260A168A11382B831203133908013A36
:10267800031D3F2B402B482BB9010A168A15C1268A
:102688000A168A11482B482B831203134008033A71
:1026980003194F2B502B192BD52AD52AD52A0A12C4
:1026A8008A111228831603171A171A1B5C2B602B22
:1026B800831203179B17632B831203179B139B1B10
:1026C800662B6A2B8312031798176D2B8312031737
:1026D8009813981B702B742B831603171417772BDA
:1026E800831603171413141B7A2B7E2B83160317D8
:1026F8001117812B831603171113111B842B882B99
:102708008312031792178B2B8312031792130A1243
:102718008A11482F9B179B1B922B962B831203170A
:102728009517992B831203179513951B9C2BA02B98
:10273800831203179817A32B831203179813981B58
:10274800A62BAA2B831603171417AD2B8316031772
:102758001413141BB02BB42B831603171117B72BA4
:10276800831603171113111BBA2BBE2B83120317E1
:102778009217C12B8312031792138B2B8B2B75087F
:10278800003A03198E2B013A0A168A1103197E2D75
:10279800033A03198E2D013A0319B82D073A031984
:1027A800E22D013A0319042E033A03192E2E013A99
:1027B8000319642E0A168A110F3A03195C2C013A80
:1027C8000319562B8B2B8B2B831603179A12831204
:1027D80003171A1114111711831603179412911263
:1027E8008312031711110A128A15022B8316031775
:1027F8009416941A002C042C831603179116072C90
:102808008316031791128B2B171517190C2C102CE4
:10281800831203171415132C831203171411141998
:10282800162C1A2C831603179A161D2C83160317B9
:102838009A129A1A202C242C831603179116272CE7
:10284800831603179112911A2A2C2E2C8312031720
:102858001115312C8312031711118B2B171517190A
:10286800362C3A2C8316031794163D2C831603171F
:102878009412941A402C442C831603179A16472C4A
:10288800831603179A129A1A4A2C4E2C831603178A
:102898009116512C831603179112911A542C582C07
:1028A8008312031711155B2C8312031711118B2B3D
:1028B8000A128A11582F1B161B1A632C672C8312B5
:1028C80003179B156A2C831203179B119B196D2CF8
:1028D800712C831203171816742C831203171812FD
:1028E800181A772C7B2C8312031715167E2C83124B
:1028F80003171512151A812C852C8312031712162B
:10290800882C831203171212121A8B2C8F2C831205
:1029180003179215922C8312031792110A128A1127
:10292800482F9B159B19992C9D2C831203179515DD
:10293800A02C8312031795119519A32CA72C831289
:1029480003171816AA2C831203171812181AAD2C7D
:10295800B12C831203171516B42C83120317151202
:10296800151AB72CBB2C831203171216BE2C831210
:1029780003171212121AC12CC52C831203179215B1
:10298800C82C831203179211922C922C7508003AC6
:102998000319952C013A0A168A110319CC2E033A09
:1029A8000319DA2E013A0319042F073A03192E2FB7
:1029B800013A03194E2F033A0319782F013A0319E4
:1029C800AC2F0A168A110F3A03197B2D013A031905
:1029D8005F2C922C922C831203171B139B129512B7
:1029E80098121513121392120A128A1581291517B3
:1029F800151BFF2C032D831203171217062D8312A4
:102A080003171213922C9816981A0B2D0F2D831258
:102A180003179516122D831203179512951A152D63
:102A2800192D831203171B171C2D831203171B1351
:102A38001B1B1F2D232D831203171217262D8312FC
:102A480003171213121B292D2D2D8312031792160B
:102A5800302D831203179212922C9816981A352D3E
:102A6800392D8312031715173C2D831203171513DD
:102A7800151B3F2D432D831203171B17462D831259
:102A880003171B131B1B492D4D2D831203171217F8
:102A9800502D831203171213121B532D572D831217
:102AA800031792165A2D831203179212922C151798
:102AB800151B5F2D632D831203171217662D8312C2
:102AC80003171213121B692D6D2D831203171B1781
:102AD800702D831203171B131B1B732D772D831265
:102AE80003179B167A2D831203179B12922C0A1236
:102AF8008A11492F831603171417141B842D882D48
:102B08008316031711178B2D8316031711130A1237
:102B18008A11482F9817981B922D962D8312031708
:102B28009517992D831203179513951B9C2DA02D8E
:102B3800831603171A17A32D831603171A131A1BC4
:102B4800A62DAA2D831603171117AD2D831603176B
:102B58001113111BB02DB42D831203179217B72D23
:102B68008312031792138B2D9817981BBC2DC02D19
:102B7800831603171417C32D831603171413141B76
:102B8800C62DCA2D831603171A17CD2D83160317C2
:102B98001A131A1BD02DD42D831603171117D72DEE
:102BA800831603171113111BDA2DDE2D8312031759
:102BB8009217E12D8312031792138B2D8316031797
:102BC8001417141BE82DEC2D831603171117EF2D7E
:102BD800831603171113111BF22DF62D83160317F5
:102BE8001A17F92D831603171A131A1BFC2D002E1A
:102BF800831203179B17032E831203179B138B2D26
:102C08009817981B082E0C2E8316031714170F2ECF
:102C1800831603171413141B122E162E831603176C
:102C28001A17192E831603171A131A1B1C2E202E77
:102C3800831203179B17232E831203179B139B1BC7
:102C4800262E2A2E8312031792172D2E831203176E
:102C580092138B2D831603171A171A1B342E382E2E
:102C68008316031714173B2E831603171413141B0C
:102C78003E2E422E831203179817452E83120317F0
:102C88009813981B482E4C2E8312031795174F2E16
:102C9800831203179513951B522E562E8312031772
:102CA8009B17592E831203179B139B1B5C2E602EB8
:102CB800831203179217632E8312031792138B2D17
:102CC800831603171417141B6A2E6E2E8316031708
:102CD8001117712E831603171113111B742E782EDA
:102CE8008312031792177B2E8312031792138B2DCF
:102CF800831603171A171A1B822E862E83120317A0
:102D08009B17892E831203179B139B1B8C2E902EC7
:102D1800831203179517932E831203179513951B88
:102D2800962E9A2E8312031798179D2E8312031737
:102D38009813981BA02EA42E831603171417A72EDA
:102D4800831603171413141BAA2EAE2E831603170B
:102D58001117B12E831603171113111BB42EB82E99
:102D6800831203179217BB2E8312031792138B2D0E
:102D7800F6000A128A112E2F831203171B129B11B9
:102D8800951118121512121292110A168A11CA2CCC
:102D98001516151AD02ED42E831203171216D72EF5
:102DA8008312031712120A128A11482F1816181ABA
:102DB800DE2EE22E831203179515E52E83120317D4
:102DC80095119519E82EEC2E831203171B16EF2E7A
:102DD800831203171B121B1AF22EF62E83120317E7
:102DE8001216F92E831203171212121AFC2E002F34
:102DF800831203179215032F831203179211D72EEC
:102E08001816181A082F0C2F8312031715160F2FD0
:102E1800831203171512151A122F162F8312031770
:102E28001B16192F831203171B121B1A1C2F202F76
:102E3800831203171216232F831203171212121A62
:102E4800262F2A2F8312031792152D2F831203176B
:102E58009211D72E1516151A322F362F83120317F3
:102E68001216392F831203171212121A3C2F402FF1
:102E7800831203171B16432F831203171B121B1AE7
:102E8800462F4A2F831203179B154D2F83120317C2
:102E98009B11D72E1816181A522F562F8312031764
:102EA8001516592F831203171512151A5C2F602F48
:102EB800831203171B16632F831203171B121B1A87
:102EC800662F6A2F831203179B156D2F8312031722
:102ED8009B119B19702F742F831203179215772F4C
:102EE800831203179211D72E1B161B1A7C2F802FC3
:102EF800831203171516832F831203171512151A39
:102F0800862F8A2F8312031718168D2F8312031703
:102F18001812181A902F942F831203179515972FAC
:102F280083120317951195199A2F9E2F8312031751
:102F38009B15A12F831203179B119B19A42FA82F50
:102F4800831203179215AB2F831203179211D72EF2
:102F58001516151AB02FB42F831203171216B72F90
:102F6800831203171212121ABA2FBE2F83120317D5
:102F78009215C12F831203179211D72E1B161B1AF5
:102F8800C62FCA2F831203179B15CD2F8312031741
:102F98009B119B19D02FD42F831203179515D72F68
:102FA8008312031795119519DA2FDE2F8312031751
:102FB8001816E12F831203171812181AE42FE82F96
:102FC800831203171516EB2F831203171512151A00
:102FD800EE2FF22F831203171216F52F8312031701
:102FE8001212121AF82FFC2F831203179215FF2FB3
:082FF800831203179211D72E7A
:103D6200F701F801B601B701B801B901BA01BB0107
:103D7200BC01BD01BE01BF0183010A168A117C2A62
:103D82008030F5003E30F600C72EC72E0130F50216
:103D92000030031CF603F602FF307606031DD32E15
:103DA200FF307506031DD62ED72EC72ED82E08003B
:103DB200F60083120313BD01BB01E92E7608F63E1D
:103DC200F5007508F6000130F5007508BD07E92E0B
:103DD2000A3076020318EE2EEF2EDF2EF02E760832
:103DE200F5007508BB0008008312031790019101CA
:103DF200920193019401950196019701980199010D
:103E02009A019B018316031790019101920193017C
:103E12009401950196019701980199019A019B01DC
:103E220090168312031790160800F501F601192F58
:103E320083120313201C1E2F1F2F252F2208F50784
:103E42000318F60A2308F60701300310A20DA30D8A
:103E5200FF3E031D262F01300310A10CA00CFF3ED4
:103E6200031D2D2F21082004031D382F392F192F50
:103E72003A2F7608A101A1077508A001A007412FDA
:103E8200080001308312031788003E309C00843002
:103E92009D00FF309E00FF30831603179C00FC300C
:103EA2009D00FF309E00DB308312031787000A1645
:103EB2008A15F5260A168A150F308312031390000D
:103EC2008316031311141118672F6B2F8316031314
:103ED20091146E2F831603139110813083120313F2
:103EE2009F00831603131F169F161F1300308312A1
:103EF2000313BC00F5007508BA000C30F500750814
:103F0200C100F801C0010314C00D83120317181772
:103F1200831603130610861706178312031306145B
:103F22008316031316179617831203130C108316A6
:103F320003130C140B108B150B178B1708000C1C9A
:103F4200A32FA42FD72F831603130C1CA92FAA2F3C
:103F5200D72F7714831203130C1080308F00013097
:103F6200F0007008BC073D303C02031CB92FBA2F89
:103F7200D72F0130F0007008BA07BC013D303A0279
:103F8200031CC42FC52FD72F0130F0007008C107C2
:103F9200BA010D304102031CCF2FD02FD72FC10100
:103FA2000314C10DD72FD72FD72FD72F0B1CDA2FE2
:103FB200DB2FF42F8B1DDE2FDF2FF42F8312B8019E
:103FC200B901061BE52FE62FEA2FB8010314B80D3D
:103FD200EA2F861BED2FEE2FF22FB9010314B90D34
:103FE200F22F0B10F42F74088312FF0073088A005B
:0E3FF20072088400710E8300FE0E7E0E090020
:02400E00D4F0EC
:00000001FF
